:10100000006000205D130000A5130000A71300007E
:10101000A9130000AB130000AD1300000000000096
:10102000000000000000000000000000AF130000FE
:10103000B113000000000000B3130000B51300005E
:10104000BD290000B7130000C92B00004931000082
:10105000B713000000000000452A0000B71300008D
:10106000B7130000B7130000B7130000B713000058
:10107000B7130000B7130000B7130000B713000048
:10108000B71300003D1E0000B7130000B7130000A7
:10109000B7130000B713000051370000B71300006A
:1010A000B7130000B71300000000000000000000AC
:1010B00049300000B71300000000000000000000ED
:1010C0000000000000000000000000000000000020
:1010D0000000000000000000000000000000000010
:1010E0000000000000000000000000000000000000
:1010F00000000000000000000000000000000000F0
:1011000000000000000000000000000000000000DF
:1011100000000000000000000000000000000000CF
:1011200000000000000000000000000000000000BF
:1011300000000000000000000000000000000000AF
:10114000000000000000000000000000000000009F
:10115000000000000000000000000000000000008F
:10116000000000000000000000000000000000007F
:10117000000000000000000000000000000000006F
:10118000000000000000000000000000000000005F
:10119000000000000000000000000000000000004F
:1011A000000000000000000000000000000000003F
:1011B000000000000000000000000000000000002F
:1011C000000000000000000000000000000000001F
:1011D000000000000000000000000000000000000F
:1011E00000000000000000000000000000000000FF
:1011F00000000000000000000000000000000000EF
:10120000354936480A1A02D0072291438D4634499F
:1012100034480A1A06D00722914381F30988022232
:1012200082F3148830483149314A00F044F831489B
:101230003149324A00F03FF831483249324A00F031
:101240003AF832483249334A00F035F832483349E7
:10125000334A00F030F833483349344A00F02BF871
:1012600033483449344A00F026F8344834490022DF
:1012700000F02CF833483449002200F027F83348B6
:101280003349091A082902DB002202604160314A11
:1012900090471F481F49884205D00268043003B4B4
:1012A000904703BCF7E700208646EC46002000216B
:1012B000294A9047FEE7884207D0521A05D00378A2
:1012C00001300B700131013AF9D17047884202D0E8
:1012D00002700130FAE770470060002000580020DB
:1012E00000600020006000208C3E0000080000200C
:1012F0003C000020EC130000EC13000060390000FB
:101300008C3E00000800002008000020443A000045
:10131000443A0000443A0000443A0000443A0000D5
:10132000443A0000443A0000443A00008C3E000079
:10133000C03E00003C0000203C0000203C0000209B
:1013400052070020540700205407002054070020B3
:10135000540F002073130000C933000000F02CB8B4
:101360000B484FF00701884385460A488047FFF73E
:1013700047BF094809490A4A884207D0521A05D08E
:10138000037801300B700131013AF9D17047000048
:101390000060002069250000443A00000800002099
:1013A00008000020FEE7FEE7FEE7FEE7FEE7FEE7B7
:1013B000FEE7FEE7FEE7FEE709480068094909681D
:1013C0000A280AD1002908D1074802686FF0700383
:1013D0001A404FF040031A430260FFF7C1BF0000FC
:0C13E0003001001034010010E40E004049
:1013EC00F0B595B01D46164608460C4601F068F857
:1013FC001A9B0D93CDE9086500252B46082205A9FB
:10140C0020460A958DF82C500C9501F075F8079B29
:10141C000293069B03939DF814308DF8115003F042
:10142C000302012A1DD1BDF81420059DC3F3C2038C
:10143C00C2F383168DF81030B20008230EA9204693
:10144C0001F05AF8C5F3952508AB0093324602AB70
:10145C000EA9284600F0DCFA204601F035F815B04C
:10146C00F0BD022AF8D1BDF81650C3F3C203C5F380
:10147C0089158DF810300827082D2E4628BF082610
:10148C003B4632460EA9204601F036F8AD1B08ABA0
:10149C0002AA31460EA8374400F01EFB002DEBD1FA
:1014AC00DAE70378024613F0040006D003F00300D9
:1014BC00012803D0022809D0012070470B6812883C
:1014CC000233C2F3831213440B6070470B685288CB
:1014DC00023303EB92130B60EEE700002DE9F04FA3
:1014EC00DFF81CA187B00F4600230446861C0DF1C3
:1014FC00070015468DF8073000F04AFCDAF8042096
:10150C003A60DAF8083003F580739B1A0AF21C472C
:10151C000AF583690AF21448B3421AD30020002D4D
:10152C0069D004F00F039B0143F0050363F30F0034
:10153C00DAF80430DAB2033233444AF822009DF868
:10154C000700CAF8043000F047FC012007B0BDE8E2
:10155C00F08F0121384600F0FAFC484600F00FFDF0
:10156C00404600F00CFDDAF808000290C0B20330DF
:10157C000AEB800002A9FFF794FF029B30BBDAB2A2
:10158C000AEB8202D16803919A1C0133DBB20AEB9D
:10159C0083030292D3F80CB001F00303012B22D089
:1015AC00022B15D08346404600F0ECFC10B1029B98
:1015BC00CAF808305946384600F0C9FCDAF8083049
:1015CC00DAF8042003F580739B1AA5E7D8B2CEE7AE
:1015DC00BDF80E30C3F3891303334FEA1B4B02EBF8
:1015EC0093030293DFE7BDF80C30C3F383134FEA88
:1015FC001B4B1344F5E7A40544F0060098E700BF25
:10160C000C01002030B50A4C71B10A4A0A49121B70
:10161C00D20800239A4201D1002030BD31F823506A
:10162C00854202D00133F5E7034654F83300F4E762
:10163C00AC390000343A000008000020094B013995
:10164C0003EBC000032909D8DFE801F00A02040605
:10165C00042070470079704740797047002070472C
:10166C0002207047AC39000070470000034BD3E9EF
:10167C000130C31A58425841704700BF0C0100207A
:10168C002DE9F04186B0FFF7F1FF0546002840F048
:10169C00ED80774CC4F81804BFF34F8FA368029306
:1016AC00DBB2033304EB830002A9FFF7FAFE029BC3
:1016BC0018B1D4F81824002A5AD0DAB2991C013384
:1016CC0004EB8202DBB204EB8303D268DB68049385
:1016DC0002F00303022B0392029154D1BDF80E3099
:1016EC006448C3F38917502F3E4628BF502606F195
:1016FC00080166F38F13C1F30901ADF80E3000F049
:10170C00B0FE0546002800F09C8000F0D9FE0023B6
:10171C00082203A9284600F0E5FE0299CB43DBB270
:10172C000133C9B20331B6EB830F4FEA830204EBEA
:10173C00810125D95FFA82F80823A6EB0806284612
:10174C0000F0D0FEF6B208F108034B4903F0FC039D
:10175C003246284600F0C6FE029B033703EB970780
:10176C000297D4F81834002B43D1D4F8106453E00A
:10177C0062689A4294D8A260284606B0BDE8F0810F
:10178C0008233246E5E7012B5BD1BDF80C30394814
:10179C00C3F38311062928BF062161F38913023193
:1017AC0001F00F018900ADF80C3000F05AFE05462F
:1017BC00002846D000F084FE0023082203A9284606
:1017CC0000F090FE0026BDF80C20C2F38312B3008B
:1017DC00964203F10803C4D202994A1CC9B20331E0
:1017EC00029204EB81010422284600F07BFE0136B4
:1017FC00E9E7284600F068FEFFF738FF80F00105A6
:10180C00EDB2B9E7F3685B7923B1336829461B68FD
:10181C0030469847F3681E68002EF3D1284600F036
:10182C0053FE0DF107008DF8076000F0B1FAD4F803
:10183C0018340BB9029BA3609DF8070000F0CCFA9A
:10184C00DAE7D4F8104454B90C4B0D480D49C01AC2
:10185C00C008000440F0020000F05EF8CCE72368FA
:10186C0020469B689847E3681C68ECE7002583E7F3
:10187C000C0100209839000018010020AC39000040
:10188C00DC390000553A00002DE9F34704460E46BA
:10189C00924601A9012218469946FFF71FFE1C4FDC
:1018AC0010B3019D4FF00008AA1CC84508EB0201BB
:1018BC0025D11848002100F01BFB80F31000000418
:1018CC0040EA1440E4006B1C04F03804DBB2EDB2C7
:1018DC0044F0010407EB8303033544EA881444EA1B
:1018EC008624D86047F825403B781BB1FFF7C8FE2B
:1018FC000028FBD1FFF7B8FE02B0BDE8F087C9B2F3
:10190C0007EB81015AF82830CB6008F10108CCE7CD
:10191C000C0100202805002000231A46FFF7B4BF55
:10192C0007B50123019201AAFFF7AEFF03B05DF8E2
:10193C0004FB000038B5084B0125D3F810441D708A
:10194C0004B938BDE3685D71236820465B6898472D
:10195C00E3681C68F4E700BF0C010020C38873B572
:10196C0004460D4633B1144A00921449144A2846D1
:10197C0000F054FB217A05291CD0637A4BB1A08866
:10198C00FFF75CFE0F4B104953F82020284600F05F
:10199C0045FB227A0D4BA08853F822600021FFF7FB
:1019AC0031FE0B4903463246284602B0BDE8704072
:1019BC0000F034BB02B070BD8A3A0000723A0000ED
:1019CC006A3A0000FC3A00008F3A0000203B00000D
:1019DC00923A000010B5037A052B0C460FD0437ACF
:1019EC0023B1084A0849204600F018FB0749204655
:1019FC0000F014FB2046BDE8104000F004BB002AA8
:101A0C00F8D0F3E78A3A00008F3A0000873A0000DA
:101A1C002DE9F04385B01F460C9D002395F80C90E2
:101A2C002B7306460C46904629463846FFF796FF20
:101A3C00B8F1060F09D8DFE808F00412181F283394
:101A4C0040003146284600F0E9FA00222946384683
:101A5C00FFF7C0FF85F80C9005B0BDE8F083226855
:101A6C003146284600F0DAFAEFE7D4E90023314694
:101A7C00284600F0D3FAE8E7A36800933146D4E98E
:101A8C000023284600F0CAFADFE7E3680193A36855
:101A9C0000933146D4E90023284600F0BFFAD4E77E
:101AAC0023690293E3680193A36800933146D4E958
:101ABC000023284600F0B2FAC7E763690393236951
:101ACC000293E3680193A36800933146D4E90023A1
:101ADC00284600F0A3FAB8E708292DE9F74F80460D
:101AEC000E4617461C463DD800251B7B2573214608
:101AFC0010460193FFF732FFDFF888A0DFF888B0BB
:101B0C00AE4232D918F805205946204600F086FA24
:101B1C000135082DF4D11D49DFF874A0DFF874B03D
:101B2C00204600F07BFA4FF000094E4524D918F8F6
:101B3C0009507E2D1ED8284601F0AAFE002814BF9D
:101B4C002A462E225946204600F068FA09F101096E
:101B5C00B9F1080FE9D1012221463846FFF73AFFC7
:101B6C00019B237303B0BDE8F08F5146204600F073
:101B7C0055FACDE72E22E5E75146204600F04EFA05
:101B8C00E4E700BFA23A00009C3A0000A63A00002D
:101B9C00A43A0000A83A0000014B01221A707047C9
:101BAC006D0500207047000070B50E4D06460FCD38
:101BBC0088B06C460FC495E80F00002E84E80F0027
:101BCC00094A0A484FF0060308BF002269460093F1
:101BDC0000F08CFE08B100F03FF8054B1E7008B009
:101BEC0070BD00BF343B0000A51B0000100000209E
:101BFC002C05002008B5044801F02EF9BDE808407A
:101C0C000020FFF7D1BF00BF1400002007B5044B24
:101C1C000093044A4023FFF7E3FB03B05DF804FB99
:101C2C00351C00002D05002010B5084C0848002379
:101C3C00D2B2237001F0ACF908B100F00DF8054BED
:101C4C001A7812B12378002BFBD010BD6D05002043
:101C5C00140000202C0500201FB50021039001AAC0
:101C6C0044F20100CDE9011101F0C0FB05B05DF8B3
:101C7C0004FB000008B50A4800F0C4F8094AD2E990
:101C8C000031C018084BD3E9002341F10001904208
:101C9C0071EB030303D210F1807041F1000108BD18
:101CAC001C000020700500208805002037B5054673
:101CBC000C460A4801A900F0C5F860B105704460F3
:101CCC0001A9064800F0E8F818B1054800F09EF8A4
:101CDC00002003B030BD0420FBE700BF78050020D6
:101CEC001C000020F7B5044600250DF1070017462F
:101CFC000E468DF8075000F04BF8D4E90223B3F1EF
:101D0C00FF3F08BFB2F1FF3F07D1FFF7B3FF301819
:101D1C0041F10001C4E9020101259DF8070000F022
:101D2C005BF855B12369A76103B1266121460020F8
:101D3C0003B0BDE8F040FFF7B9BF284603B0F0BDD3
:101D4C0037B5054600240DF107008DF8074000F06B
:101D5C001FF8D5E90223B3F1FF3F08BFB2F1FF3FF3
:101D6C0006D04FF0FF324FF0FF33C5E902230124B8
:101D7C009DF8070000F030F834B12946012003B07B
:101D8C00BDE83040FFF792BF204603B030BD0000E5
:101D9C0070B5EFF3108672B60C4A946801239CB9A7
:101DAC0093600B4B0B4DD3F8801029401160C3F896
:101DBC008050D3F8841051604FF0FF32C3F8842068
:101DCC00047006B962B670BD0370FAE79005002086
:101DDC0000E100E0FC06FFBD084B9A6810B55AB153
:101DEC0050B9EFF3108172B6054A1C6814605C6838
:101DFC005460986001B962B610BD00BF9005002018
:101E0C0000E100E00368D3F80405704790F9043052
:101E1C00002B09DB5A09012103F01F0301FA03F31C
:101E2C004032024941F82230704700BF00E100E027
:101E3C00024B034A1B681068184700BFA40500201A
:101E4C009C05002037B550E8013F9DB2C48925445C
:101E5C008489A54228BF2D1B0489A54202BFBFF36C
:101E6C002F8F002207E0C5EA030540E80154002C3F
:101E7C00E9D14FF001028DF803200193019A0A6019
:101E8C009DF8031001F0FF0321B1006810FA82F0F5
:101E9C0003B030BD1846FBE70A884B889A4209D13B
:101EAC0050E8012FC2EA024240E80123002BF7D18F
:101EBC00012070470020704701F01F024B090121DF
:101ECC00914000EB830000F01EB801F01F030122CB
:101EDC009A404B0900EB8300D14300F02CB84B091E
:101EEC0001F01F0150F82300C84000F001007047BA
:101EFC0010B5034653E8000F0A4643E8002494F05B
:101F0C00000FF7D110BD10B5034653E8002F42EA7D
:101F1C00010043E8000494F0000FF6D110BD10B599
:101F2C00034653E8000F00EA010243E8002494F052
:101F3C00000FF6D110BD10B5034653E8002F02EA8E
:101F4C00010043E8000494F0000FF6D110BD10B569
:101F5C00034653E8002F02EB010043E8000494F021
:101F6C00000FF6D110BD10B5034653E8002FA2EBBD
:101F7C00010043E8000494F0000FF6D110BD0121DC
:101F8C00FFF7C1BF0021FFF7CABF37B505460024D4
:101F9C000DF107008DF80740FFF7FAFE2A686B6811
:101FAC00116899420ED9481E106011F8013CEC687A
:101FBC00298A01FB0344AB6811791B1ADBB29942E5
:101FCC0038BF13719DF80700FFF706FF204603B0DA
:101FDC0030BD37B5054600230DF107000C468DF8D2
:101FEC000730FFF7D5FE2A681368591C1160E968A1
:101FFC00641A298AB4FBF1F41C709DF80700FFF7F2
:10200C00EBFE03B030BD826810B504462AB14369BB
:10201C000168006998470023A36010BD0EB403B596
:10202C00039921B104AB01AA019300F077F802B037
:10203C005DF804EB03B070470A2938B504460D4629
:10204C0002D10D21FFF7F8FFA3682268591CA1608B
:10205C00D554D4E901329A4204D32046BDE8384025
:10206C00FFF7D1BF38BD00002DE9F84F9846DDE9E8
:10207C000A43154682460F460A464FF00109AA420A
:10208C000FD2C14538BFC14613F0010B01D16CB959
:10209C0000240126B8F1010F1BD908F1FF386E435B
:1020AC00F8E709F10109B2FBF5F2E8E79B070ED559
:1020BC00B8F1000F0CBF30262026A145E9D2013C17
:1020CC0031465046FFF7B8FF002CF6D1E0E720264A
:1020DC00F3E7B7FBF6F39D42E1D9DFF83C80B7FBA1
:1020EC00F6F3504618F8031006FB1377FFF7A4FF1E
:1020FC003346AB42B6FBF5F6F1D2BBF1000F02D082
:10210C000CB1A14501D3BDE8F88F20215046013C0C
:10211C00FFF792FFF4E700BF753B00002DE9F74F86
:10212C00054617468846002900F03E8118F8011B29
:10213C0049B92B7B002B00F03781284603B0BDE852
:10214C00F04FFFF760BF252940F0B780002698F8C4
:10215C0000302D2B424608F1010823D0302B24D01F
:10216C002B2B25D000242A2B02F1010123D13B6813
:10217C001A1D1B683A601C440A4613782E2B26D174
:10218C0001324FF0000A104610F8011BA1F1300C7F
:10219C00BCF1090F1DD80A2303FB0A13A3F1300A63
:1021AC000246F0E746F00106D1E746F00206CEE71C
:1021BC0046F00406CBE711F8013CA3F130000928E6
:1021CC00DBD80A2202FB0434303C0A46CBE74FF042
:1021DC00000A12F8011B01F0FB0068289046F8D0A9
:1021EC00782909D86F290CD8632962D022D82529DF
:1021FC0063D0582900F0888098F80030002B95D1D6
:10220C0097E770390829F7D801A353F821F000BFDC
:10221C008F2300000522000005220000252300006A
:10222C000522000003230000052200000522000007
:10223C0015230000642901D06929DDD13A68D2F850
:10224C000090111D89EAE9723960A2EBE9724FF036
:10225C00010B092A35DCD34538BFD3462CB1B9F173
:10226C00000F01DB720700D5013CB30702D5BAF1B0
:10227C00000F03D0F00701D44CBB0024B9F1000FC0
:10228C002DDAC9F100092D212846FFF7D5FE06F0FD
:10229C000302022A04D1BAF1000F01D11CBB0024A5
:1022AC00CDE9004653460A2249462846FFF7DCFE94
:1022BC00A2E73B681A1D19783A602846FFF7BCFE66
:1022CC009AE70A230BF1010BB2FBF3F2C1E7A3452A
:1022DC00D4D220212846013CFFF7AEFECCE7710793
:1022EC00D5D52B21D0E7A345DAD230212846013CA5
:1022FC00FFF7A2FED2E73968CDE900460A1D3A6025
:10230C0053460A220968D0E739680A1D3A60CDE9BC
:10231C00004653461022F5E73B681A1D3A6016F04A
:10232C000106D3F8009024D1B9F1000F03D0484630
:10233C0001F0DFFA0646B4421DD809F1FF3919F84D
:10234C00011F00293FF458AF2846FFF775FEF6E74A
:10235C0028460136FFF770FE19F806100029F7D150
:10236C00A642BFF449AF20212846013CFFF764FE8A
:10237C00F6E70026F0E720212846013CFFF75CFE3B
:10238C00D9E73B681A1D3A60302128461C68FFF7D4
:10239C0053FE78212846FFF74FFE00220823CDE993
:1023AC0000322146102280E703B0BDE8F08F00BF59
:1023BC002DE9F84FB0F806A04579D2F800B09DF899
:1023CC0028900AFB05F5043D88460BEB0301A94256
:1023DC0003F1040488BFA5EB030BB4FBFAF6074624
:1023EC000AFB1644C2F800B04EB9AAEB04055D45D1
:1023FC0028BF5D46BBF1000F04D1BDE8F88F3F68E4
:10240C00013EF1E7043408EB06003C442A46B9F1DE
:10241C00000F0DD02146ABEB050B01F041FADA456C
:10242C002E443F6855464FF0000428BF5D46E1E757
:10243C0001462046EFE7F8B546790146721E05467F
:10244C00002393422D6803D30024A64202D8F8BD82
:10245C000133F6E70F682846FFF7BBFD0134394618
:10246C00F3E72DE9F843068ACD1C0746FFF78DFDEF
:10247C00043E35440446B5FBF6F5F0B14FF48073D9
:10248C00EDB28380C680013D076081464FF00008A5
:10249C00A84512D23846FFF778FD064648B1637955
:1024AC000133637108F10108C9F800000760814627
:1024BC00EEE72046FFF7BFFF34462046BDE8F88321
:1024CC0001210430FFF743BD10B50121044604304F
:1024DC00FFF749FDC0B220B92046BDE81040FFF718
:1024EC00AABF10BD1FB503920022009203AAFFF7EA
:1024FC005FFF05B05DF804FB1FB50392012200924B
:10250C0003AAFFF755FF05B05DF804FB0B684A689A
:10251C004360934208BF0023016008BF43607047CB
:10252C00436843B10268916852680B44934243601C
:10253C0004BF0023436070474FF08053D3F8300141
:10254C00A0F10A035842584170470000024AD2F8E1
:10255C000034002BFBD0704700E0014010B5FFF7B2
:10256C00EBFF48B14FF080534FF08042D3F8443228
:10257C00C3F34233C2F83C35FFF7DEFF40B14FF0F6
:10258C0080430022C3F80C21C3F81021C3F838256E
:10259C00FFF7D2FF002846D04FF08052494BD2F8BB
:1025AC000414C3F82015D2F80814C3F82415D2F873
:1025BC000C14C3F82815D2F81014C3F82C15D2F843
:1025CC001414C3F83015D2F81814C3F83415D2F813
:1025DC001C14C3F84015D2F82014C3F84415D2F8D3
:1025EC002414C3F84815D2F82814C3F84C15D2F8A3
:1025FC002C14C3F85015D2F83014C3F85415D2F873
:10260C003414C3F86015D2F83814C3F86415D2F832
:10261C003C14C3F86815D2F84014C3F86C15D2F802
:10262C004424C3F87025FFF787FF48B14FF080436F
:10263C00D3F80024D20744BF6FF00102C3F8002482
:10264C004FF08053D3F830210A2A0AD1D3F8343111
:10265C003BB14FF08042D2F8E43E43F00F03C2F896
:10266C00E43E4FF01023D3F80022002A03DBD3F80A
:10267C000432002B22DA144901234FF01020C1F848
:10268C0004351524FFF762FFC0F80042FFF75EFF28
:10269C00C0F80442FFF75AFF0023C1F80435FFF7D6
:1026AC0055FFBFF34F8F0949094BCA6802F4E0622A
:1026BC001343CB60BFF34F8F00BFFDE7054B064ABA
:1026CC001A6010BD00C0004000E0014000ED00E0C9
:1026DC000400FA05240000200090D003044B1A5C7F
:1026EC00012393404FF0A042C2F80835704700BF59
:1026FC00973B000008B50020FFF7F0FF0120FFF723
:10270C00EDFF0220FFF7EAFFBDE808400320FFF7CA
:10271C00E5BF0000074A4FF0A041105CD1F804352A
:10272C000122824022EA03001340C1F80805C1F8D7
:10273C000C357047973B0000C20708B501460CD515
:10274C004FF0A0430322C3F84427C3F84827C3F82B
:10275C004C27C3F85027FFF7CDFF8B070AD54FF056
:10276C00A0430C22C3F83427C3F83827C3F83C27FE
:10277C00C3F8402708BD000038B5074C051E04F10E
:10278C00080318BF1C4623682BB11A6822605B68CB
:10279C0028469847F7E738BDB005002020B9054B0F
:1027AC0001225A70FFF7E8BF012802D1014A90704C
:1027BC00F8E77047A805002020B9034B01225A7096
:1027CC00FFF7DABF704700BFA805002038B50E4CE4
:1027DC002378B3B90D486360A3602361E36000F014
:1027EC00B7F8054600F094FF08B900F0BDF80123D6
:1027FC002370074BD3F800340BB10123A370284688
:10280C0038BD8525F5E700BFA8050020A9270000E5
:10281C000000014037B50D4C00230DF107008DF879
:10282C000730FFF7B5FAE368013BE360E36833B9BF
:10283C00074BD3F8005415B900F0A8F8A5709DF813
:10284C000700FFF7C9FA03B030BD00BFA805002090
:10285C0000000140012813B50CD0032820D038B952
:10286C00134B0122C3F88020BFF34F8FBFF36F8F40
:10287C0002B010BD0F4C00230DF107008DF807308E
:10288C00FFF786FA23780BB9FFF7A0FFE3689DF8F2
:10289C0007000133E3600123A370FFF79DFAE7E71C
:1028AC0000F062F802B0BDE81040FFF7B3BF00BF04
:1028BC0000E100E0A80500201FB503788DF800307A
:1028CC004368019383688DF80830C368054A039305
:1028DC00054B684653F8213052F82110984705B043
:1028EC005DF804FBBC050020C0050020F0B50646D1
:1028FC000F4B16F804CB43F82C200E4B17460C4606
:10290C000A6943F82C200FCC89B06D460FC594E8AA
:10291C000F00002F85E80F00074ACDF810C008BF44
:10292C003A466946304600F0D5F909B0F0BD00BF13
:10293C00C0050020BC050020C528000000F1804027
:10294C00002382B0036003680193019B02B07047BF
:10295C00044B0246187918B91A6001229A80704704
:10296C0085207047C4050020074B1A68D20704D491
:10297C00C02283F8002301221A604FF08043012209
:10298C00C3F81825704700BF00E100E04FF080420B
:10299C0008B50223C2F808334FF48270FFF7CEFF5C
:1029AC000123D360D2F81834DB03FBD408BD00003C
:1029BC004FF0804110B5D1F8003163B14FF4807005
:1029CC00FFF7BCFF0D4B58790122C1F8082310B951
:1029DC005A711B6898474FF08042D2F8043163B1AA
:1029EC004FF48270FFF7AAFF0223C2F80833034B9F
:1029FC00BDE810401B680120184710BDC40500201D
:102A0C0000F1804000F5C040002382B003600368F1
:102A1C000193019B02B07047800000F1A040D0F8F8
:102A2C00002722F44032C0F80027D0F8003743EAE0
:102A3C000143C0F8003770472DE9F74F00244E4D85
:102A4C0001944FF48072012102F1804303F5C043DD
:102A5C0090B21B68012B06D1D5F804330B4202D07F
:102A6C00FFF7CEFF0C430432B2F5907F4FEA4101E1
:102A7C00EAD1414BD3F87C31012B0CD14FF4BE7011
:102A8C00FFF7BEFF4FF0A04344F00044D3F82025DD
:102A9C000192C3F82025E3B2D3B1384F00250126AB
:102AAC00344210D0AB0003F1804303F5C043D3F89C
:102ABC001005D3F8101557F8253023B1C1F3014197
:102ACC00C0F3042098470135082D4FEA4606E7D19C
:102ADC00002C48DA294D4FF0A048294E4FF0000940
:102AEC00012716F9013B5A1C31D0C3F3C20208323C
:102AFC006A44DCB212F8042C03F03F0A03F007031B
:102B0C0007FA03F31A4222D00AF5E073504658F83C
:102B1C002330C3F3014BBBF1020F0CBF0321022185
:102B2C00FFF77AFF07FA0AF3C8F8203505EB0A031A
:102B3C0093F9303055F823304BB1A109032904D057
:102B4C00BBF1020F12D1012901D15046984709F16E
:102B5C000109B9F1040FC4D1D8F820350193C8F894
:102B6C002035002BB9D103B0BDE8F08FBBF1030FBA
:102B7C00EDD10229E8E700BF00600040CC05002041
:102B8C001C0600200020704770470023435082B081
:102B9C0043580193019B02B0704700001FB50123FD
:102BAC008DF80030044BCDE90110D3E900126846D2
:102BBC00904705B05DF804FB280600207FB5434A1A
:102BCC00D2F82461002E60D010464FF49271FFF7BA
:102BDC00DCFF02238DF80030D2F88034C2F8803448
:102BEC000393D2F83C350293394BDA6801920022F8
:102BFC00C3E906226846D3E9001290473348D0F85F
:102C0C00443173B14FF4A271FFF7BFFF304B9A6997
:102C1C003AB10022C3E90622D968D0F83C05FFF787
:102C2C00BDFF2A48D0F82031ABB14FF49071FFF7BB
:102C3C00ACFF0123C360264B5A6962B1D0F84C1526
:102C4C000291002299688DF8002001915A61684622
:102C5C00D3E9001290471D48D0F858319BB14FF47E
:102C6C00AC71FFF792FF1A4B5A6962B1D0F84C1550
:102C7C000291002299688DF8002001915A616846F2
:102C8C00D3E90012904704B070BDD2F81031002B7C
:102C9C00B4D04FF488711046FFF777FF0C4BD2F885
:102CAC003C0599698842A9D1DC69D96864B1D2F82C
:102CBC00005225F02005C2F800521A699C61DA60B6
:102CCC00DE61FFF76BFF99E79C61FAE7002000409B
:102CDC00280600202DE9F8435A4E90F8048024234E
:102CEC0003FB0863044693F820300D469146002BF5
:102CFC0040F0A38054490068FFF744FF07460028C2
:102D0C0040F09D802A682068511C0BD04FF0A041E8
:102D1C0001239340C1F8083502F5E0734FF0030C22
:102D2C0041F823C069684B1C1FBF01F5E0734FF0DD
:102D3C00A04C4FF0000E4CF823E0AB69C0F82435E2
:102D4C0095F814C06B7DBCF1010F4CEA0303C0F87D
:102D5C006C35C0F80C25C0F814151DD1AA68531C8D
:102D6C001FBF02F5E0734FF0A0414FF0000C41F88B
:102D7C0023C0EB68591C0BD04FF0A04C012199409B
:102D8C00CCF8081503F5E0714FF0030E4CF821E078
:102D9C00C0F80835C0F81025242202FB08F2B3183D
:102DAC00C3F804902B69B350B9F1000F2FD04FF436
:102DBC0088712A7FFFF7E9FE20684FF49071FFF7C6
:102DCC00E4FE20684FF49271FFF7DFFE20684FF4A9
:102DDC00A271FFF7DAFE4FF4AC712068FFF7D5FE55
:102DEC0023681A49C3F80413190B43F30733520130
:102DFC00002BD2B21CDB1648C51885F80023012223
:102E0C005B0901F01F0102FA01F140F8231023685D
:102E1C000822C3F80025242303FB08660023C6E917
:102E2C0006337361012386F820303846BDE8F883F9
:102E3C00084B01F00F015A54E9E70827F5E7112771
:102E4C00F3E700BF28060020C92B00001003420046
:102E5C0000E100E014ED00E0F8B5444C05792423C2
:102E6C0003FB054302465B680068ABB1404BC0F8FE
:102E7C00083340F30733002B4FEA10310CDB01F021
:102E8C001F065B090121B14020333A4E46F823104E
:102E9C00BFF34F8FBFF36F8FD0F8003223F02003B6
:102EAC00C0F80032242303FB05439B692BB14FF47C
:102EBC00A271FFF76AFE012343604FF4AC71FFF778
:102ECC0064FE0123C360242303FB0543D0F858118F
:102EDC000029FBD0996919B1D0F844110029F5D01B
:102EEC000023C0F800351368D3F80C75D3F81465BB
:102EFC00D3F80825D3F810154FF0FF3C6745C3F8FD
:102F0C000CC518BF07F5E077C3F814C5C3F808C59E
:102F1C00C3F810C51EBF4FF0A0434FF0020C43F88E
:102F2C0027C0771C1FBF4FF0A04306F5E0760227A1
:102F3C0043F826704E1C1FBF01F5E0714FF0A04303
:102F4C00022643F82160531C1FBF4FF0A04302F52B
:102F5C00E072022143F82210FFF716FE242303FB34
:102F6C000544002384F820306360F8BD2806002057
:102F7C001003420000E100E00279044B242101FB24
:102F8C0002335869003818BF01207047280600200A
:102F9C0001F06043B3F1005F2DE9F0470646884627
:102FAC0092463BD190F80490FFF7E6FF04460028C8
:102FBC0036D11D4F3068242505FB09754FF49071EF
:102FCC00C5F814A0C5F80880FFF7DFFD4FF4AC710D
:102FDC003068FFF7DAFD33686A69A968C3F84415ED
:102FEC00C3F8482501229A606A68DAB9D3F820211F
:102FFC00D3F858011AB90028F8D00F2007E00028A0
:10300C00FBD10122DA60D3F85821002AFBD024230B
:10301C0003FB097700237B61BDE8F0871020FBE7F9
:10302C001120F9E72046F7E728060020002343503B
:10303C0082B043580193019B02B070472148D0F8ED
:10304C00103110B55BB14FF48871FFF7EFFF1E4BD9
:10305C005A79510703D51B680BB1012098471948C1
:10306C00D0F814315BB14FF48A71FFF7DFFF164BC8
:10307C005A79120703D51B680BB1022098471148E7
:10308C00D0F81C315BB14FF48E71FFF7CFFF0E4BB4
:10309C00587910F0100002D11B6803B19847094809
:1030AC00D0F8043163B14FF48271FFF7BFFF064BC8
:1030BC0001221A711B681BB1BDE810400320184790
:1030CC0010BD00BF00C001404C060020002343503F
:1030DC0082B043580193019B02B070470A7B0346B0
:1030EC00032A29D8DFE802F0212519028A68500347
:1030FC0004D5D3F84C250869904207D18A6852034D
:10310C001AD4D3F84C254969914215D000200622D7
:10311C00C3F80005C3F800257047D3F84C2508699F
:10312C009042F3D1D3F83C25EDE7D3F84C2509694F
:10313C00EAE7D3F83C25FAE701207047F0B5594D82
:10314C00594CD5F8243187B0FBB14FF49271284615
:10315C00FFF7BCFFD5F80431BBB9A368C5F8083339
:10316C000223A360A368C5F80433D5F860311BB102
:10317C00D5F800329F0503D44A4B01221A625A61DA
:10318C00012384F82E3007B0F0BDD5F80431002BA4
:10319C0050D044484FF48271FFF798FF236A5E06C3
:1031AC0009D494F82E3033B93F49FFF797FF80F0DC
:1031BC00010084F82E00236A5D0720D43B4E0FCE0D
:1031CC0001AD0FC5336837482B604FF4B071FFF772
:1031DC007DFF4FF4AE71FFF779FF94F8303013B1E7
:1031EC0094F82E305BB12F4B0022C3F80022A26062
:1031FC002F4AC3F808232F4B0822C3F88021294AF1
:10320C00D2F8C434C2F8C43498073DD501238DF8E4
:10321C00003094F830300BB984F82F30236A5B07F8
:10322C0003D594F82E30002BADD0D4E9003168468C
:10323C009847A8E71B484FF4A471FFF747FF237B7F
:10324C0083B91A4F0FCF01AE0FC63B68336094F8A9
:10325C003030002BD3D1C5F80032A360144BC5F825
:10326C000833C8E74FF40073C5F8003240F202236C
:10327C00A36003F1CE73C5F80833A368C5F8043313
:10328C000123AB602B627EE7590701D50223BEE711
:10329C00DA0701D50323BAE794F82E30002BB6D009
:1032AC000423B4E7003000405406002060060020E0
:1032BC0002029C0100E100E0032811D8012A0AD186
:1032CC0001290FD100F10E02D2B20D4B00EB4000E0
:1032DC001A54002070470129F7D0022904D049B1B3
:1032EC00072070470022F8E7054B00EB400018441C
:1032FC004270EEE7024B00EB400018448270E8E7A6
:10330C008806002008B5012202210020FFF7D4FF17
:10331C0008B1072810D1072202210120FFF7CCFFAA
:10332C0008B1072808D100210A220846FFF7C4FF7C
:10333C0010B1072808BF002008BD00000388102B1F
:10334C0010B502D0112B1ED010BD1A4C2168B1B98A
:10335C0001220846FFF7B0FF08B1072824D1072245
:10336C0002210120FFF7A8FF08B107281CD1042275
:10337C0002210020FFF7A0FF08B1072814D1236811
:10338C0001332360E0E70B4A1368013B1360002B09
:10339C00DAD1FFF7B7FF0028D6D0074B1B68002BFC
:1033AC00D2D0BDE810401847034B1B68002BE6D069
:1033BC009847E4E7980600209406002070B5012099
:1033CC00094DFFF7B9F945F0010500242046FFF738
:1033DC00A1F94FF4FA764FF47A40A847013EFAD19E
:1033EC000134042CF2D1F0E7D03B000008B50546BF
:1033FC0072B6FEF79FFAFEF743F90028FBD1114B8A
:10340C00114C1249E41AE4082A462404104D44F0E5
:10341C000100FEF785FAD5F8F030DB0700D500BEC9
:10342C000C4944F00200FEF777FABFF34F8FEA68BD
:10343C00094B02F4E0621343EB60BFF34F8F00BF04
:10344C00FDE700BFAC390000DC390000D63B0000C2
:10345C0000ED00E0E53B00000400FA05034B1A8880
:10346C0082420CBF18460020704700BFB8060020EF
:10347C00024B9B6903B11847704700BF9C060020A4
:10348C0013B50B46497A02460E4871B9D0E90110C2
:10349C001C7A002C18BF01465868FEF723FC78B143
:1034AC0002B0BDE81040FFF7E3BF00211972436979
:1034BC0033B101218DF80410ADF8062001A898470E
:1034CC0002B010BD9C0600204B8802889A4212D88C
:1034DC0042889A420FD380888B8840F2F31188423D
:1034EC0094BF021A421A9A4205D80844984234BF33
:1034FC000020012070470020704700000388122B29
:10350C0070B5014659D004D8102B1ED0112B44D0C5
:10351C0070BD502BFCD12F4BC288DB899A42F7D15E
:10352C00038A022BF4D186883046FFF797FF0546B5
:10353C000028EDD001F1120000F0E6F838BB686805
:10354C00FEF7FEFB0028E3D009E0C37B012BDFD1A3
:10355C004FF6FF70FFF782FF054620B90420BDE847
:10356C007040FFF785BF1C4A8E88068000230372CB
:10357C001368C0F80A305368C0F80E3010310A30A6
:10358C00FFF7A2FF134B6872DB89002BC0D12946D1
:10359C003046BDE87040FFF773BF8088FFF75EFFD1
:1035AC0004460028B4D04068FEF7CAFB08B1FFF708
:1035BC005FFF4FF6FF732380AAE786883046FFF73C
:1035CC004DFF05460028A3D008310A30FFF77CFFD9
:1035DC006872DCE79C060020CC0600200AB1FEF7DE
:1035EC006BBCFEF772BC73B50191019C06466CB1C5
:1035FC0000252C46294601A8FEF771FC18B106EBF4
:10360C00440301349D800135142DF3D130463460D0
:10361C0002B070BD2DE9F04303888488103B8DB057
:10362C000A2B1ED8DFE803F006361D1D1D1D1D1DBF
:10363C001D5B3D002E4FBB68DB43009379686846E9
:10364C00FEF779FC009901A8FFF7CDFF0DF10808F2
:10365C000026019B9E4207D3132C12D90420FEF79F
:10366C00FBFA0DB0BDE8F08338F8029B002501355C
:10367C00494607EB8500FEF728FC1E2DF7D10136D5
:10368C00E7E721461B48FEF717FC1B482146FEF7CF
:10369C0013FCE6E7174821460DB0BDE8F043FEF7F2
:1036AC0014BC027A15483F2A4FEA1215214694BFE2
:1036BC0000220122FFF792FF022D94BF002201226B
:1036CC000F482146FFF78AFF012D0E4894BF0022B8
:1036DC00012221460DB0BDE8F043FFF77FBF037A0E
:1036EC00002BBED1427A0548C2F3C0022146F1E755
:1036FC00D4060020DC060020D8060020EC060020B2
:10370C00E8060020E4060020008800F00100704765
:10371C00014B1878704700BF5007002007B50849C7
:10372C006846FEF7F3FE019B13B903B05DF804FB8A
:10373C00D3E9002090476846FEF7F2FEF3E700BF9E
:10374C00103C0000FFF7EABF61DF704730B5134D46
:10375C00ADF5017D4FF4FA740DF1020103A8ADF83B
:10376C000240FFF7F1FF70B9294601A8FEF7CEFE23
:10377C00029B002BF0D003A8D3E90021904701A8AD
:10378C00FEF7CEFEF4E7052805D00DF5017DBDE86A
:10379C003040FEF761BA0DF5017D30BD283C0000CC
:1037AC00024B1B780BB1FFF7D1BF704751070020BC
:1037BC004BDF70471FB50E4C01A8FFF7F9FF70B92E
:1037CC00214602A8FEF7A2FE039B002BF4D0019821
:1037DC00D3E90021904702A8FEF7A2FEF4E70528E2
:1037EC0004D004B0BDE81040FEF736BA04B010BDEA
:1037FC00403C00007F2805D8034A044B105C5B5CFE
:10380C001840704700207047583C0000D83C00001E
:10381C00A0F16103192B98BF20387047A0F1410328
:10382C00192B98BF203070477F299ABF0170012057
:10383C006FF02E00704700BF5AB10A787F2A0AD861
:10384C0000B102600021501AC3E9001118BF012019
:10385C007047104670476FF02E007047A0F161035F
:10386C00192B98BF20387047A0F14103192B98BF32
:10387C00203070477F2805D8034A044B105C5B5CF2
:10388C001840704700207047583C0000D83C00009E
:10389C00024B5B689B6809211B68184728000020B5
:1038AC00844640EA010313F0030F18D18446202A02
:1038BC000BD32DE9F007B1E8F807A0E8F807A2F15F
:1038CC002002202AF7D2BDE8F007042A07D351F8CA
:1038DC00043B40F8043BA2F10402042AF7D2002A6C
:1038EC0005D011F8013B00F8013B013AF9D16046D3
:1038FC00704700F1010110F0030F11D010F8012BEB
:10390C00002A23D010F0030F0AD010F8012B002A44
:10391C001CD010F0030F03D010F8012B002A15D087
:10392C002DE970004FF001324FF0803350F8044B0A
:10393C00A4EB020525EA04051D4000D1F6E7A0F131
:10394C00040070BC10F8012B002AFBD1A0EB010085
:04395C0070470000B0
:08396000C52700000000000073
:10396800213600000000000049330000000000007C
:08397800093500000000000009
:083980006128000000000000B6
:10398800AD37000000000000C13700000000000053
:103998003C000020040100200C010020440000200D
:0439A8001800000003
:1039AC00A13B000000000000A73B0000000000004D
:1039BC00AE3B000000000000B83B0000000000001F
:1039CC00BC3B000000000000B23B00000000000007
:1039DC00663A000000000303603B0000000000009A
:1039EC006B3B000000000000FF3B000000000000EB
:1039FC009B3B000000000000F23B000000000303B2
:103A0C00073C0000000003031C3C00000000030303
:103A1C00343C000000000303853B00000000000064
:083A2C008E3B000000000000C9
:103A3400543B000000000000443A0000080000204D
:103A4400756172745F6C6F675F6261636B656E64EE
:103A5400004261636B656E647320666C75736865A0
:103A64006400617070001B5B313B33316D00257362
:103A74004C6F67732064726F7070656420282564CE
:103A84002925730D0A001B5B306D002573003C254E
:103A9400733E2025733A2000202530327800202000
:103AA40020007C002563001B5B313B33306D001B21
:103AB4005B313B33326D001B5B313B33336D001B99
:103AC4005B313B33346D001B5B313B33356D001B85
:103AD4005B313B33366D001B5B313B33376D006527
:103AE40072726F72007761726E696E6700696E66DA
:103AF4006F006465627567008A3A0000AB3A0000A3
:103B04006A3A0000B33A0000BB3A0000C33A00002E
:103B1400CB3A0000D33A0000DB3A0000000000007A
:103B2400E33A0000E93A0000F13A0000F63A0000F6
:103B3400FFFFFFFFFFFFFFFFFFFFFFFFFFFFFFFF91
:103B440000000000000000000000D6010600000094
:103B5400191C0000011C0000B11B00006170705FA3
:103B6400627574746F6E006170705F74696D6572F4
:103B740000303132333435363738394142434445E5
:103B8400467077725F6D676D7400736F72746C69E1
:103B940073740011121314636C6F636B00434C4F06
:103BA400434B004750494F54450050525300554130
:103BB4005254450050574D005457494D00000000E1
:103BC4000000000000000000000000000738FDD8DD
:103BD4007047466174616C206572726F722025694A
:103BE4000053797374656D207265736574006E7229
:103BF400665F626C655F6761747400626C655F6EBA
:103C04007573006E72665F73646800008839000023
:103C140098390000080000006E72665F7364685F84
:103C2400626C6500683900008039000008000000FB
:103C34006E72665F7364685F736F6300603900005F
:103C4400683900000800000043000000504F534949
:103C54005800000020202020202020202068282830
:103C64002828202020202020202020202020202040
:103C740020202020481010101010101010101010C8
:103C840010101010848484848484848484841010A8
:103C940010101010108181818181810101010101C5
:103CA40001010101010101010101010101010110F1
:103CB400101010101082828282828202020202029A
:103CC40002020202020202020202020202020210C2
:103CD4001010102000070320041702010857104099
:103CE400800000004C3C0000503D0000643E000099
:103CF40053756E004D6F6E00547565005765640012
:103D04005468750046726900536174000000000035
:103D14004A616E00466562004D6172004170720036
:103D24004D6179004A756E004A756C0041756700F3
:103D3400536570004F6374004E6F760044656300F2
:103D440000000000414D00504D000000883E00007E
:103D5400843E0000843E0000843E0000843E000057
:103D6400843E0000843E0000843E0000843E000047
:103D7400843E0000FFFFFFFFFFFFFFFFFFFFFFFF89
:103D8400FFFF0000C43D0000F43C0000003E0000C2
:103D9400143D0000483D0000A83D0000583E0000CE
:103DA400B43D0000256D2F25642F25790000000007
:103DB40025612025622025652025542025590000F1
:103DC40053756E646179004D6F6E6461790054754A
:103DD4006573646179005765646E65736461790025
:103DE400546875727364617900467269646179001C
:103DF4005361747572646179000000004A616E75E4
:103E0400617279004665627275617279004D617202
:103E1400636800417072696C004D6179004A756E87
:103E240065004A756C790041756775737400536554
:103E34007074656D626572004F63746F62657200C1
:103E44004E6F76656D62657200446563656D62658B
:103E54007200000025483A254D3A25530000000021
:103E6400013800001D3800002938000081380000A6
:103E74006938000075380000353800004538000006
:083E8400000000002E00000008
:103E8C0000000000FF0000000000000000200040C7
:103E9C000000000000100140110004000090D0034D
:103EAC00E83C0000E83C0000E83C0000E83C000076
:043EBC00E83C0000DE
:040000030000135D89
:00000001FF
